:100000000C94CD010C94FE010C94FE010C94FE01A5
:100010000C94FE010C94FE010C94FE010C94FE0164
:100020000C94FE010C94FE010C94FE010C94FE0154
:100030000C94FE010C94FE010C94FE010C94FE0144
:100040000C94FE010C94FE010C94FE010C94FE0134
:100050000C94FE010C94FE010C94FE010C9477109C
:100060000C94FE010C944D100C9423100C94FE0182
:100070000C94FE010C94FE010C94FE010C94FE0104
:100080000C94FE010C94FE010C94FE010C94FE01F4
:100090000C94F90F0C94CF0F0C94FE010C94FE01FC
:1000A0000C94FE010C94FE010C94FE010C94FE01D4
:1000B0000C94FE010C94FE010C94FE010C94FE01C4
:1000C0000C94FE010C94FE010C94FE010C94A50FFF
:1000D0000C947B0F0C94FE010C94FE010C94FE0119
:1000E0000C94FE010C9432070C941B0E0C94140714
:1000F0000C94A7020C949F0D0C9404160C940C0EF7
:100100000C9493140C941B170C94C20D0C94D205F0
:100110000C94F60D0C944C040C94200E0C943E029E
:100120000C9456040C9419060C9464060C94ED146B
:100130000C944E030C9404170C945A070C9430043E
:100140000C94DB140C9468140C94B90D0C94B50247
:100150000C94CA050C94DE0D0C943A040C941A0706
:100160000C9411040C9477160C94CB0D0C94160E71
:100170000C9449170C9490150C949E070C94480409
:100180000C9424070C94C1100C94EB050C9493026E
:100190000C94C6070C945A060C94F5050C9474073D
:1001A0000C9426040C94040E0C94E1050C947A161D
:1001B0000C9432160C942C040C9475140C941704A3
:1001C0000C9484020C94B00D0C94D40D0C949207F2
:1001D0000C94DE140C94FD0D0C94FD050C94440756
:1001E0000C94C4140C9401030C94E80D0C94571552
:1001F0000C94A80D0C9444040C94960D0C94460693
:100200000C9436040C943E040C9423060C942304A2
:100210000C941B040C9432060C940F160C9451048D
:100220000C940F060C94EF0D0C943C060C945204A5
:100230000C9405060C948C0D0C941F040C9437142C
:100240000C94D7050C9450060000210024002700D0
:100250002A002D00300033000101000004010701D5
:100260000A0100002200250028002B002E0031008A
:10027000340002010000050108010B01000020000C
:100280002300260029002C002F003200000100006E
:100290000301060109010505050507050808080809
:1002A000020202020A0A080804040404010101010E
:1002B0000101010103030303030303030407070709
:1002C0000C0C0C0C0C0C0C0C0202020206060606AE
:1002D000060606060B0B0B0B0B0B0B0B0A0A0A0A86
:1002E0000A0A08080707050505040404010210208E
:1002F000200808102040102040800201020108045C
:1003000002010102040810204080804020100804EF
:100310000201800402018040201008040201080448
:10032000020101020408102040800102040810208C
:100330004080040810204080048008100440801091
:10034000204000000A0B02090C0D0E0807030401EF
:10035000000000000000000000000000000000009D
:10036000000000000000000000000000000012116A
:10037000100000000000000000000000000000006D
:10038000000000000000000000000000000000006D
:100390000000000000000000C11011241FBECFEFBC
:1003A000D1E2DEBFCDBF00E00CBF13E0A0E0B2E0C1
:1003B000ECEAF6E300E00BBF02C007900D92AC340C
:1003C000B107D9F726E0ACE4B3E001C01D92AA3032
:1003D000B207E1F711E0CDECD1E000E006C02197D3
:1003E0000109802FFE010E944C1BCC3CD10780E00C
:1003F0000807A9F70E943A110C94541B0C940000B2
:100400000F931F93CF93DF93EC019A01AB01E8891F
:10041000F98982E08083EC85FD8510820E851F8539
:1004200060E874E88EE190E00E94CB182150310919
:10043000410951095695479537952795F80120832D
:10044000188EEC89FD8986E08083EA89FB898081AA
:1004500080618083EA89FB89808188608083EA8962
:10046000FB89808180688083EA89FB8980818F7D18
:100470008083DF91CF911F910F910895AF92BF922A
:10048000CF92DF92EF92FF920F931F93CF93DF9360
:100490006C017B018B01040F151FEB015E01AE188F
:1004A000BF08C017D10759F06991D601ED91FC91B1
:1004B0000190F081E02DC6011995892B79F7C501CE
:1004C000DF91CF911F910F91FF90EF90DF90CF9030
:1004D000BF90AF900895FC01A089B1898C91A68945
:1004E000B78982FD0FC09C91818D8F5F8F73228DA4
:1004F000821749F0A18DAE0FBF2FB11D5D969C9361
:10050000818F08958C910895FC01538D448D252F82
:1005100030E0842F90E0821B930B541710F0CF969D
:10052000089501970895FC01918D828D981761F0CF
:10053000A28DAE0FBF2FB11D5D968C91928D9F5FE6
:100540009F73928F90E008958FEF9FEF0895FC01C5
:10055000918D828D981731F0828DE80FF11D858D78
:1005600090E008958FEF9FEF0895FC01918D228D0B
:10057000892F90E0805C9F4F821B91098F73992790
:10058000089583E394E00E94B50221E0892B09F4E9
:1005900020E0822F089580ED94E00E94B50221E0D2
:1005A000892B09F420E0822F08958DE695E00E94C2
:1005B000B50221E0892B09F420E0822F0895FC0187
:1005C000A48DA80FB92FB11DA35ABF4F2C91848DB4
:1005D00090E001968F739927848FA689B7892C9311
:1005E000A089B1898C91837080648C93938D848D64
:1005F000981306C00288F389E02D80818F7D808367
:100600000895EF92FF920F931F93CF93DF93EC0126
:1006100081E0888F9B8D8C8D98131AC0E889F989A9
:10062000808185FF15C09FB7F894EE89FF896083AC
:10063000E889F98980818370806480839FBF81E02D
:1006400090E0DF91CF911F910F91FF90EF9008956F
:10065000F62E0B8D10E00F5F1F4F0F731127E02E4A
:100660008C8D8E110CC00FB607FCFACFE889F98982
:10067000808185FFF5CFCE010E94DF02F1CFEB8DA7
:10068000EC0FFD2FF11DE35AFF4FF0829FB7F89456
:100690000B8FEA89FB8980818062CFCFCF93DF9374
:1006A000EC01888D8823B9F0AA89BB89E889F9898A
:1006B0008C9185FD03C0808186FD0DC00FB607FCBF
:1006C000F7CF8C9185FFF2CF808185FFEDCFCE01F2
:1006D0000E94DF02E9CFDF91CF910895EF92FF9260
:1006E0001F93CF93DF9380917703811176C0809120
:1006F000760381112DC083E394E00E94B502049734
:100700000CF46BC083E394E00E94930280938C030B
:1007100083E394E00E94930280938D0383E394E04B
:100720000E94930280938E0383E394E00E949302DD
:1007300080938F0399279C012C5F3F4F3093750363
:10074000209374030297439700F581E0809376032A
:1007500083E394E00E94B502E0907403F090750387
:1007600097012450310982179307B8F114E0C12F83
:10077000D0E0CE15DF05E8F483E394E00E94930215
:10078000C457DC4F88831F5FF2CF83E394E00E945D
:10079000B502892B11F183E394E00E9493028091CA
:1007A0007203909173030196909373038093720385
:1007B000ECCF83E394E00E94B502892B29F083E318
:1007C00094E00E949302F5CF84E080937703109227
:1007D00076031092730310927203DF91CF911F91F1
:1007E000FF90EF9008958150823108F05AC0E82FB1
:1007F000F0E08827E150FC4F8F4F0C944C1B1F04F6
:100800002304110417041B04510426042C0430048F
:1008100036043A043E044404480451044C0452048F
:100820005604809180008F77809380000895809196
:1008300080008F7DF9CF80918000877FF5CF84B5D0
:100840008F7784BD089584B58F7DFBCF8091B000F4
:100850008F778093B00008958091B0008F7DF9CF9D
:10086000809190008F778093900008958091900000
:100870008F7DF9CF80919000877FF5CF8091A00088
:100880008F778093A00008958091A0008F7DF9CF8D
:100890008091A000877FF5CF809120018F77809392
:1008A00020010895809120018F7DF9CF8091200152
:1008B000877FF5CFCF93DF93282F30E0F901EE5BF0
:1008C000FC4F8491F901E451FD4FD491F901EA56AE
:1008D000FD4FC491CC23A1F081110E94F303EC2FB2
:1008E000F0E0EE0FFF1FE458FD4FA591B491EC919D
:1008F000ED2381E090E009F480E0DF91CF9108954D
:1009000080E090E0FACF1F93CF93DF93282F30E061
:10091000F901EE5BFC4F8491F901E451FD4FD49154
:10092000F901EA56FD4FC491CC23A9F0162F81118D
:100930000E94F303EC2FF0E0EE0FFF1FEE59FD4F86
:10094000A591B4918FB7F894EC91111108C0D0958E
:10095000DE23DC938FBFDF91CF911F910895DE2BB3
:10096000F8CFCF93DF9380918B03823009F44DC091
:10097000833009F465C081112FC080ED94E00E949E
:10098000B50203974CF180ED94E00E94A7028E37E8
:10099000910581F580ED94E00E94930280ED94E052
:1009A0000E94930280ED94E00E94A702079739F419
:1009B00080ED94E00E94930282E080938B0380EDAF
:1009C00094E00E94A7024D9751F480ED94E00E94BC
:1009D000930283E080938B03DF91CF91089580EDA4
:1009E00094E00E94B502892BB9F380ED94E00E9457
:1009F0009302F5CF80ED94E00E94B502892B61F35C
:100A000080ED94E00E949302F5CF80ED94E00E9487
:100A1000B50208970CF3C8E0D8E080ED94E00E949E
:100A20009302D0938B03C150C1F780ED94E00E94F4
:100A3000B502892B89F280ED94E00E949302F5CFF4
:100A400061E08AE10E94830480ED94E00E94B50297
:100A50004E9714F2CEE1D4E080ED94E00E94930230
:100A6000D0938B03C150C1F780ED94E00E94B50292
:100A7000892B09F4B1CF80ED94E00E949302F4CF6A
:100A800080E090E0892B29F00E94D50281110E941C
:100A900000000E94CB0281110E94B1040E94C10299
:100AA00081110E946E0380E090E0892B49F080E084
:100AB00090E0892B29F00E94000081110C94000025
:100AC0000895CF93DF9390E0FC01E451FD4F249112
:100AD0008A569D4FFC0184918823D1F090E0880FC5
:100AE000991FFC01E85BFD4FA591B491FC01EE5903
:100AF000FD4FC591D49161110EC09FB7F8948C91B0
:100B0000E22FE0958E238C932881E223E8839FBF18
:100B1000DF91CF9108958FB7F894EC91E22BEC938D
:100B20008FBFF6CF1F93CF93DF93182FEB0161E0B8
:100B30000E946105209739F460E0812FDF91CF9109
:100B40001F910C948304CF3FD10511F461E0F5CFE0
:100B5000E12FF0E0EE5BFC4FE491E150E23108F070
:100B6000B3C0F0E08827E854FA4F8F4F0C944C1B29
:100B7000CA05D205D705E105EB056406F505FD05B7
:100B800005060F061906230632063C0664064606CD
:100B900050065A0684B5806884BDC7BDDF91CF91E9
:100BA0001F91089584B5806284BDC8BDF7CF809140
:100BB0008000806880938000D0938900C093880073
:100BC000EDCF80918000806280938000D0938B0075
:100BD000C0938A00E3CF809180008860809380007A
:100BE000D0938D00C0938C00D9CF8091B0008068E5
:100BF0008093B000C093B300D1CF8091B0008062E9
:100C00008093B000C093B400C9CF809190008068F9
:100C100080939000D0939900C0939800BFCF8091AB
:100C20009000806280939000D0939B00C0939A00C4
:100C3000B5CF80919000886080939000D0939D0004
:100C4000C0939C00ABCF8091A00080688093A000EF
:100C50008091A0008F7B8093A000D093A900C093C7
:100C6000A8009CCF8091A00080628093A000D093C8
:100C7000AB00C093AA0092CF8091A00088608093BF
:100C8000A000D093AD00C093AC0088CF809120012C
:100C9000806880932001D0932901C09328017ECFE2
:100CA00080912001806280932001D0932B01C0931A
:100CB0002A0174CF80912001886080932001D09315
:100CC0002D01C0932C016ACFC038D1050CF03ECF66
:100CD00033CF863308F0865320917B00982F98708D
:100CE000277F922B90937B008770806480937C0099
:100CF00080917A00806480937A0080917A0086FDEA
:100D0000FCCF809178009091790008953FB7F894D6
:100D10008091810390918203A0918303B091840319
:100D200026B5A89B05C02F3F19F00196A11DB11D46
:100D30003FBFBA2FA92F982F8827BC01CD01620F82
:100D4000711D811D911D43E0660F771F881F991F3C
:100D50004A95D1F708958091E6039091E703A09119
:100D6000E803B091E903813E9E42A105B10520F060
:100D700089E080937F0309C08091FC039091FD037B
:100D800080359105C0F410927F03E0917F03EA3033
:100D900008F002C1F0E08827EF52F94F8F4F0C9412
:100DA0004C1BC60714071A072407320744075A07C3
:100DB00074079E0792079C0120553109243631059E
:100DC00010F481E0D6CF9C01245B31092436310533
:100DD00010F482E0CECF9C012851314024363105F9
:100DE00010F483E0C6CF9C012C57314024363105E6
:100DF00010F484E0BECF9C01205E314024363105E2
:100E000010F485E0B6CF9C012454324024363105DD
:100E100010F486E0AECF885A92408436910510F4E3
:100E200087E0A7CF88E0A5CF61E085E20E94830438
:100E300060E005C061E085E20E94830461E084E235
:100E40000E94830460E009C061E085E20E9483049F
:100E500061E084E20E94830461E083E20E948304F3
:100E600060E00DC061E085E20E94830461E084E2FD
:100E70000E94830461E083E20E94830461E082E2D5
:100E80000E94830460E011C061E085E20E94830457
:100E900061E084E20E94830461E083E20E948304B3
:100EA00061E082E20E94830461E081E20E948304A7
:100EB00060E015C061E085E20E94830461E084E2A5
:100EC0000E94830461E083E20E94830461E082E285
:100ED0000E94830461E081E20E94830461E080E279
:100EE0000E94830460E019C061E085E20E948304EF
:100EF00061E084E20E94830461E083E20E94830453
:100F000061E082E20E94830461E081E20E94830446
:100F100061E080E20E94830461E08FE10E9483042B
:100F200060E029C080917D0390917E03833091051C
:100F30002CF5019690937E0380937D0361E085E21A
:100F40000E94830461E084E20E94830461E083E202
:100F50000E94830461E082E20E94830461E081E2F6
:100F60000E94830461E080E20E94830461E08FE1DB
:100F70000E94830461E08EE10C9483048630910525
:100F80003CF4019690937E0380937D0360E04DCF07
:100F900010927E0310927D03089560E089E00E9424
:100FA000830480918603843009F463C030F488237D
:100FB00081F0813091F10C94AB06863009F47EC04B
:100FC00008F475C08730B9F71092F10310928603C8
:100FD000F2CF8091E3038130D1F0809126044091DB
:100FE000FC035091FD032091290430912A04840FC1
:100FF000952F911D2817390708F4C901883C9105E0
:1010000010F488EC90E090937C0380937B0381E064
:10101000809386038093E303CECF8091FC0390916D
:10102000FD0320917B0330917C0328173907D8F00A
:101030002091290430912A0428173907A0F08091C3
:101040000A0490910B04883E934068F48091E60373
:101050009091E703A091E803B091E903803E9E429E
:10106000A105B10520F085E080938603A4CF84E03C
:10107000FBCF609115046093D8038091FC0390919D
:10108000FD0320917B0330917C032817390740F042
:101090002091290430912A0470E02817390710F4B0
:1010A00070E060E085E00E94920587E0DDCF70E0AF
:1010B00060E085E00E94920586E0D6CF70E060E0B7
:1010C00085E00E94920580917A0390911604891719
:1010D00040F087E0809386031092E30310927A0336
:1010E0006ACF8F5F80937A0366CF70E060E085E01F
:1010F0000E94920580918503813099F030F0823012
:1011000031F18630E1F10C94AB068091E30381303C
:1011100031F48093850382E08093E303F4CF82E08F
:10112000F8CF61E089E00E94830480917903909177
:1011300017048917E8F060E089E00E9483041092A8
:10114000F1031092790386E080938503DCCF61E0A0
:1011500089E00E948304809179032091FC033091FF
:10116000FD03283C310540F090911804891718F7C9
:101170008F5F80937903C7CF90911904DACF809164
:10118000780390911604891738F01092F1031092A9
:10119000850310927803B7CF8F5F80937803B3CF26
:1011A000DB01EC91F0E0E050FE4FE081E927F0E058
:1011B000E050FE4F908189278C930895FC010190A7
:1011C0000020E9F73197AF01481B590BBC018DE6B0
:1011D00095E00C943E028F929F92AF92BF920F9334
:1011E0001F93CF93DF93CDB7DEB7A1970FB6F894D7
:1011F000DEBF0FBECDBF19A2423008F44AE08E0117
:101200000F5D1F4F842E912CB12CA12CA5019401B0
:101210000E94CB18E62FB901CA01EA30F4F4E05D70
:10122000D801EE938D01232B242B252B79F790E009
:1012300080E0109719F0CD010E94DE08A1960FB64C
:10124000F894DEBF0FBECDBFDF91CF911F910F91FC
:10125000BF90AF909F908F900895E95CE1CFEF929F
:10126000FF920F931F93CF93DF937C018B010E941A
:10127000B518D82FD801EC91F0E0E050FE4FE08196
:10128000C82FCE27CC93C70101960E94B518EC2F2A
:10129000F0E0E050FE4F90819827F80190832D2FC9
:1012A00030E0322F2227820F932F911DDF91CF91B3
:1012B0001F910F91FF90EF900895CF93DF931F92AE
:1012C0001F92CDB7DEB71A8281E08983BE016F5FBE
:1012D0007F4F90E080E00E942F098230910508F056
:1012E00060C190932C0480932B04BE016F5F7F4FED
:1012F00082E090E00E942F09853323E0920708F0F6
:1013000055C190932A0480932904BE016F5F7F4FDB
:1013100084E090E00E942F09853323E0920708F0D3
:1013200048C19093280480932704BE016F5F7F4FCC
:1013300086E090E00E942F099FEF980F983C08F0FC
:101340003DC180932604BE016F5F7F4F88E090E02F
:101350000E942F09873222E0920708F031C1909352
:10136000250480932404BE016F5F7F4F8AE090E0E4
:101370000E942F09873222E0920708F024C190933F
:10138000230480932204BE016F5F7F4F8CE090E0C6
:101390000E942F09893823E1920708F017C1909322
:1013A000210480932004BE016F5F7F4F8EE090E0A8
:1013B0000E942F09893823E1920708F00AC190930F
:1013C0001F0480931E04BE016F5F7F4F80E190E099
:1013D0000E942F09893522E0920708F0FDC0909302
:1013E0001D0480931C04BE016F5F7F4F82E190E07B
:1013F0000E942F09893522E0920708F0F0C09093EF
:101400001B0480931A04BE016F5F7F4F84E190E05C
:101410000E942F09853608F0E5C080931904BE01AB
:101420006F5F7F4F86E190E00E942F098B3008F0BC
:10143000DBC080931804BE016F5F7F4F88E190E0AE
:101440000E942F09853108F0D1C080931704BE0196
:101450006F5F7F4F8AE190E00E942F09853608F088
:10146000C7C080931604BE016F5F7F4F8CE190E090
:101470000E942F0980931504BE016F5F7F4F8EE19C
:1014800090E00E942F09813127E2920708F0B2C054
:101490009093140480931304BE016F5F7F4F80E22A
:1014A00090E00E942F099093120480931104BE01D2
:1014B0006F5F7F4F82E290E00E942F0990931004AB
:1014C00080930F04BE016F5F7F4F84E290E00E9423
:1014D0002F0990930E0480930D04E981F0E0E05011
:1014E000FE4F80818983BE016E5F7F4F86E290E070
:1014F0000E942F099981981709F44CC010922C046E
:1015000010922B0426E232E030932A04209329041F
:10151000109228041092270492E39093260444EF3B
:1015200051E05093250440932404509323044093A6
:10153000220448E755E0509321044093200448E0FA
:1015400057E050931F0440931E0430931D042093D2
:101550001C0428EC30E030931B0420931A0494E11F
:101560009093190492E0909318049AE090931704D2
:101570009EE19093160490E59093150420ED37E0DA
:10158000309314042093130428E93AE330931204AF
:101590002093110480930C040F900F90DF91CF9152
:1015A000089510922C0410922B049FCE86E292E0B4
:1015B000A8CE1092280410922704B7CE82E3C1CEA1
:1015C00084EF91E0CCCE84EF91E0D9CE88E795E02E
:1015D000E6CE88E097E0F3CE86E292E000CF88EC9A
:1015E00090E00DCF84E119CF82E023CF88E02DCFAA
:1015F0008EE137CF80ED97E04BCFFF920F931F9393
:10160000CF93DF93F82E8B01EA01E881F0E0E05000
:10161000FE4F808189278883692FC8010E94BD18E9
:10162000E881F0E0E050FE4F80818F2588836F2DA8
:10163000C8010196DF91CF911F910F91FF900C94FB
:10164000BD18CF93DF931F92CDB7DEB781E08983BA
:10165000AE014F5F5F4F70E060E080912B0490918E
:101660002C040E94FD0AAE014F5F5F4F62E070E004
:101670008091290490912A040E94FD0AAE014F5FD7
:101680005F4F64E070E080912704909128040E94ED
:10169000FD0A80912604AE014F5F5F4F66E070E067
:1016A00090E00E94FD0AAE014F5F5F4F68E070E07E
:1016B00080912404909125040E94FD0AAE014F5FA1
:1016C0005F4F6AE070E080912204909123040E94B1
:1016D000FD0AA895AE014F5F5F4F6CE070E080910E
:1016E0002004909121040E94FD0AAE014F5F5F4FDC
:1016F0006EE070E080911E0490911F040E94FD0A2C
:10170000AE014F5F5F4F60E170E080911C049091EB
:101710001D040E94FD0AAE014F5F5F4F62E170E061
:1017200080911A0490911B040E94FD0A8091190473
:10173000AE014F5F5F4F64E170E090E00E94FD0AF0
:10174000A89580911804AE014F5F5F4F66E170E08D
:1017500090E00E94FD0A80911704AE014F5F5F4F39
:1017600068E170E090E00E94FD0A80911604AE01ED
:101770004F5F5F4F6AE170E090E00E94FD0A809148
:101780001504AE014F5F5F4F6CE170E090E00E9486
:10179000FD0AAE014F5F5F4F6EE170E08091130470
:1017A000909114040E94FD0AAE014F5F5F4F60E20A
:1017B00070E080911104909112040E94FD0AA89596
:1017C000AE014F5F5F4F62E270E080910F04909135
:1017D00010040E94FD0AAE014F5F5F4F64E270E0AB
:1017E00080910D0490910E040E94FD0AE981F0E0C1
:1017F000E050FE4F80818983AE014F5F5F4F66E20C
:1018000070E090E00E94FD0A0F90DF91CF91089563
:10181000CF938091E503882321F08091E403811127
:101820000DC08091710390911604981798F481E08F
:101830008093E5038093E403109271038091770312
:101840008130E9F058F08430C9F1853009F430C2B4
:10185000CF9108958F5F80937103F0CF60E089E1AD
:101860000E94830460E08AE10E94830460E08CE1CE
:101870000E94830460E08DE1CF910C9483048091F9
:101880008A038F5F823018F480938A03E1CF10922D
:101890008A0361E089E10E94830460E08AE10E949A
:1018A00083041092770383E394E00E94B502892BAE
:1018B00079F283E394E00E949302F5CF20917403C0
:1018C00030917503B90162507109FB01E457FC4F77
:1018D000808190E0982F882725573C4FD9012C9183
:1018E000820F911D50E040E0E0E02E2F30E02617FF
:1018F000370740F424573C4FD9012C91420F511D1A
:10190000EF5FF3CF8417950709F0C7C1C0918C032F
:10191000CC2311F0C23159F480918E03883409F43C
:1019200098C170F4803101F1853409F4BEC061E0E2
:1019300089E10E94830461E08AE10E94830481C0FE
:101940008A3409F499C18C3491F760E089E10E94EE
:10195000830461E08AE10E948304C23109F071C00E
:1019600081E0809389036DC060E089E10E94830477
:1019700061E08AE10E9483048091900390E0982FB7
:10198000882720919103820F911D9093DE0380930D
:10199000DD0380919203282F30E0322F222780919F
:1019A0009303820F932F911D9093CD038093CC03CB
:1019B0009C01205531092931314008F048C034E6F6
:1019C000389FA001399F500D11245093CD034093AF
:1019D000CC038091940390E0982F88272091950361
:1019E000820F911D389FA001399F500D11245093F3
:1019F000CF034093CE0380919A0390E0982F8827DD
:101A000040919B03480F592F511DEFE080919C039B
:101A100090E0982F882720919D03820F911DE89FC9
:101A2000B001E99F700D1124E49F9001E59F300DF6
:101A300011242617370708F49B013093E003209305
:101A4000DF0385E08093770310928A0301CF8054EF
:101A50009F4181369D46A8F78091940390E0982F8E
:101A6000882720919503820F911D9093CF03809337
:101A7000CE0360919A03862F90E0982F882760917B
:101A80009B03680F792F711D90E080E00E940F1A70
:101A900020E030E040EC5FE30E94C61A0E94E019AB
:101AA0007093E0036093DF03CCCF60E089E10E9494
:101AB000830461E08AE10E948304C23111F681E06F
:101AC0008093880320919103822F90E0982F88279C
:101AD00020919203280F392F311DE0919003ED5191
:101AE000E33108F5F0E08827E758F24F8F4F0C9468
:101AF0004C1B8C0D960D9F0DA80DB00DB90DC20D90
:101B0000CB0DD40DDE0DE80DEF0DF60DFD0D040E21
:101B10000C0E160E1B0E200E2230310520F43093D1
:101B20002C0420932B040E94210B8BCF2533F3E050
:101B30003F07C8F730932A0420932904F4CF2533B4
:101B400043E0340780F73093280420932704EBCF39
:101B5000C9010197883C910530F720932604E3CF13
:101B6000273282E03807F8F63093250420932404C6
:101B7000DACF2732A2E03A07B0F63093230420935D
:101B80002204D1CF2938B3E13B0768F63093210412
:101B900020932004C8CF2938E3E13E0720F6309394
:101BA0001F0420931E04BFCF2935F2E03F0708F041
:101BB000BACF30931D0420931C04B5CF293542E0E1
:101BC000340708F0B0CF30931B0420931A04ABCF36
:101BD0002536310508F0A7CF20931904A4CF2B3068
:101BE000310508F0A0CF209318049DCF2531310591
:101BF00008F099CF2093170496CF2536310508F0C9
:101C000092CF209316048FCF2F3F310511F008F0AB
:101C10008ACF2093150487CF213187E2380708F057
:101C200082CF30931404209313047DCF3093120499
:101C30002093110478CF3093100420930F0473CFB6
:101C40002436310508F46FCF30930E0420930D0431
:101C50006ACF60E089E10E94830461E08AE10E942A
:101C60008304C23109F0EDCE81E08093E503109248
:101C7000E40380938703E5CE60E089E10E9483045A
:101C800061E08AE10E948304C23109F0DACE109249
:101C9000E50381E08093E403ECCF61E089E10E94F9
:101CA000830460E08AE10E94830410927703D0CD20
:101CB000309188038091890381114AC03111E2C0BB
:101CC00010924C0382E180934D0380E180934E0398
:101CD00087E080934F038091FC039091FD039093E4
:101CE0005003809351038091F003809352038091BD
:101CF000EA03809353038091E20380935403ECE45E
:101D0000F3E090E080E020E03191830F911D2F5FA0
:101D10002930D1F7909355038093560361E08CE10D
:101D20000E94830461E08DE10E94830440914F038F
:101D300050E04C5F5F4F6CE473E083E394E00E94FB
:101D40003E021092770383E394E00E944E038ECD0F
:101D500010924C0382E180934D038CE480934E03F8
:101D600081E280934F0380912B04809350038091F4
:101D7000290490912A0490935103809352038091F7
:101D800027049091280490935303809354038091E7
:101D90002604809355038091240490912504909308
:101DA00056038093570380912204909123049093CB
:101DB00058038093590380912004909121049093BB
:101DC0005A0380935B0380911E0490911F049093AB
:101DD0005C0380935D0380911C0490911D0490939B
:101DE0005E0380935F0380911A0490911B0490938B
:101DF0006003809361038091190480936203809152
:101E00001804809363038091170480936403809186
:101E10001604809365038091150480936603809176
:101E20001304909114049093670380936803809146
:101E30001104909112049093690380936A03809136
:101E40000F049091100490936B0380936C03809126
:101E50000D0490910E0490936D0380936E03ECE457
:101E6000F3E090E080E020E04191840F911D2F5F2E
:101E70002332D1F790936F038093700310928903FC
:101E8000332309F110924C0382E180934D0382E4E5
:101E900080934E0384E080934F031092500386E5B5
:101EA00080935103ECE4F3E090E080E020E0319196
:101EB000830F911D2F5F2630D1F7909352038093AB
:101EC00053031092880380918703882309F426CF57
:101ED00010924C0382E180934D0382E480934E0381
:101EE00082E080934F031092500386E58093510364
:101EF0001092870313CF1F920F920FB60F921124E7
:101F00000BB60F922F933F934F935F936F937F93F3
:101F10008F939F93AF93BF93EF93FF9383E394E0EB
:101F20000E94DF02FF91EF91BF91AF919F918F913E
:101F30007F916F915F914F913F912F910F900BBEC9
:101F40000F900FBE0F901F9018951F920F920FB613
:101F50000F9211240BB60F922F933F934F935F93E1
:101F60006F937F938F939F93AF93BF93EF93FF9361
:101F700083E394E00E946B02FF91EF91BF91AF91D8
:101F80009F918F917F916F915F914F913F912F9191
:101F90000F900BBE0F900FBE0F901F9018951F92C1
:101FA0000F920FB60F9211240BB60F922F933F93FF
:101FB0004F935F936F937F938F939F93AF93BF9351
:101FC000EF93FF9380ED94E00E94DF02FF91EF9189
:101FD000BF91AF919F918F917F916F915F914F9141
:101FE0003F912F910F900BBE0F900FBE0F901F903F
:101FF00018951F920F920FB60F9211240BB60F92E5
:102000002F933F934F935F936F937F938F939F9300
:10201000AF93BF93EF93FF9380ED94E00E946B0228
:10202000FF91EF91BF91AF919F918F917F916F91B0
:102030005F914F913F912F910F900BBE0F900FBE6C
:102040000F901F9018951F920F920FB60F921124A8
:102050000BB60F922F933F934F935F936F937F93A2
:102060008F939F93AF93BF93EF93FF938DE695E08C
:102070000E94DF02FF91EF91BF91AF919F918F91ED
:102080007F916F915F914F913F912F910F900BBE78
:102090000F900FBE0F901F9018951F920F920FB6C2
:1020A0000F9211240BB60F922F933F934F935F9390
:1020B0006F937F938F939F93AF93BF93EF93FF9310
:1020C0008DE695E00E946B02FF91EF91BF91AF9179
:1020D0009F918F917F916F915F914F913F912F9140
:1020E0000F900BBE0F900FBE0F901F9018951F9270
:1020F0000F920FB60F9211242F933F938F939F93BC
:10210000AF93BF938091C8039091C903A091CA0374
:10211000B091CB033091800326E0230F2D3758F583
:102120000296A11DB11D209380038093C803909354
:10213000C903A093CA03B093CB038091810390910C
:102140008203A0918303B09184030196A11DB11D68
:102150008093810390938203A0938303B0938403BD
:10216000BF91AF919F918F913F912F910F900FBE93
:102170000F901F90189529E8230F0396A11DB11DFC
:10218000D2CFE3E3F4E01382128248EE53E060E042
:1021900070E0448355836683778384E093E0918382
:1021A000808325ED30E03587248724ED30E03787C4
:1021B000268720ED30E0318B208B21ED30E0338B12
:1021C000228B22ED30E0358B248B26ED30E0378BEF
:1021D000268B118E128E138E148EE0EDF4E0138296
:1021E00012824483558366837783918380832DECA9
:1021F00030E0358724872CEC30E03787268728ECC1
:1022000030E0318B208B29EC30E0338B228B2AECB1
:1022100030E0358B248B2EEC30E0378B268B118E03
:10222000128E138E148EEDE6F5E013821282448333
:102230005583668377839183808385EC90E09587CF
:10224000848784EC90E09787868780EC90E0918B80
:10225000808B81EC90E0938B828B82EC90E0958B6D
:10226000848B86EC90E0978B868B118E128E138E6A
:10227000148E0895CF93DF931F92CDB7DEB7789475
:1022800084B5826084BD84B5816084BD85B582607B
:1022900085BD85B5816085BD80916E00816080932C
:1022A0006E00109281008091810082608093810095
:1022B00080918100816080938100809180008160A5
:1022C000809380008091B10084608093B100809100
:1022D000B00081608093B000809191008260809313
:1022E0009100809191008160809391008091900095
:1022F0008160809390008091A10082608093A10012
:102300008091A10081608093A1008091A0008160F4
:102310008093A000809121018260809321018091AF
:10232000210181608093210180912001816080934F
:10233000200180917A00846080937A0080917A00F5
:10234000826080937A0080917A008E7F80937A00F9
:1023500080917A00806880937A001092C10040E0FA
:1023600052EC61E070E08DE695E00E94000282E1AF
:1023700093E00E94DE0886E293E00E94DE080E945D
:1023800086064B015C01E0E1CE2EE7E2DE2EE12C79
:10239000F12C0E948606681979098A099B09683E12
:1023A000734081059105A8F321E0C21AD108E10824
:1023B000F10838EE830E33E0931EA11CB11CC1144A
:1023C000D104E104F10429F710922E041092D403F1
:1023D0001092D5031092D6031092D70310922F04B7
:1023E0001092300410923104109232041092C603FD
:1023F0001092C703279A15B860E086E10E94610534
:1024000060E087E10E94610560E088E10E9461056B
:1024100040E855E260E070E08DE695E00E94000241
:1024200040E855E260E070E080ED94E00E94000238
:1024300040E855E260E070E083E394E00E9400022F
:10244000789461E089E00E94610561E085E00E9486
:10245000610561E085E20E94610561E084E20E941D
:10246000610561E083E20E94610561E082E20E9411
:10247000610561E081E20E94610561E080E20E9405
:10248000610561E08FE10E94610561E08EE10E94DB
:1024900061058091B100887F81608093B100809157
:1024A0009100887F8160809391001092F1031092D7
:1024B0008603109285031092D0031092D1031092DC
:1024C000D2031092D3031092D9031092DA03109220
:1024D000DB031092DC031092EF031092E3031092DF
:1024E000E6031092E7031092E8031092E90361E01B
:1024F00089E10E94610561E08AE10E94610561E075
:102500008CE10E94610561E08DE10E9461051092FD
:102510008B0310928A03109289031092880381E042
:102520008093E5038093E4031092870340E855E22B
:1025300060E070E083E394E00E9400020E945D0985
:102540000E945D090E94210BA895ECE8F3E084EB62
:1025500093E011928E179F07E1F783E991E0909342
:102560000E0480930D040E94210B89E293E00E94E7
:10257000DE086091290470912A0490E080E00E94B6
:102580000F1A2AE037ED43E25CE30E94C61A6B01A2
:102590007C01AC019B010E94331B882309F4A7C076
:1025A0008FE393E00E94DE0886E293E00E94DE085B
:1025B00040E1942E5AE0852E64E6E62EF12C76EC6E
:1025C000C72E73E0D72E0E94860600912F0410912B
:1025D0003004209131043091320460177107820772
:1025E000930708F4B9C52B013C01401A510A620A4D
:1025F000730A93018201003117422105310508F465
:102600008FC160932F0470933004809331049093B2
:1026100032047090C7030091C60310E058015FEFC9
:10262000A51AB50A87E0A822BB24000F111F36E0C7
:10263000432E82E0471408F4D6C00E946906F801D0
:10264000EA54FC4F91838083A092C60373947092E6
:10265000C7038091FE0381110BC08091FC03909110
:10266000FD039093FB038093FA0381E08093FE03C4
:102670008091F203811103C081E08093F203E09125
:10268000F103EC3208F031C1F0E08827E55BFC4E45
:102690008F4F0C944C1B371468149314C414DB1420
:1026A00075147514751475147514DE14ED14751401
:1026B0007514751457159015751475147514041642
:1026C0000F16321675147514751475147514751467
:1026D00075147716751475147514751475147514AE
:1026E0007514751475147A1604171B1749172FEFF4
:1026F0003FEF4FE75FE7C701B6010E94331B81112F
:102700000DC02FEF3FEF4FE75FE7C701B6010E9413
:10271000691918161CF483E493E044CF2FEF3FEFC0
:102720004FE75FE4C701B6010E94C11A18161CF4F6
:1027300087E493E037CF2FEF3FEF4FE75FECC70120
:10274000B6010E94691987FDF3CF2AE037ED43EA0D
:102750005BE3C701B6010E94FD184B015C010E94BA
:10276000E0196B017C010E940F1A9B01AC01C501AD
:10277000B4010E94FC184B015C014AE0C701B6019C
:102780000E94EB086EE28DE695E00E94010320E0D6
:1027900030E040E251E4C501B4010E94C61A4B0189
:1027A0005C010E94E0196B01F12CE12C4AE0C701A9
:1027B000B6010E94EB08C701B6010E940F1A9B01E7
:1027C000AC01C501B4010E94FC1820E030E040E2F9
:1027D00051E40E94C61A0E94E01990E080E04AE0AD
:1027E0000E94EB08E1CE0E946906F801EA54FC4F12
:1027F00091838083A092C6036091B4037091B50366
:10280000E6EBF3E081919191680F791FCE16DF0618
:10281000C9F793E0769567959A95E1F76C3971055C
:1028200048F41092FD031092FC031092B50310922D
:10283000B4030FCF90E080E00E940F1A27E03FE53D
:1028400048E15CE30E94C61A2DEC3CEC4CE85FE3E7
:102850000E94FC1820E030E048EC52E40E94C61AC6
:102860000E94E0197093FD036093FC03DECF80911A
:102870000804811127C060E089E00E94830481E0A0
:102880008093F1031092F0031092EF031092EB0388
:102890001092EC031092ED031092EE038091FC0372
:1028A0009091FD038834934050F070E060E085E043
:1028B0000E9492050E9475088FE08093EA030E94AF
:1028C000AB0613C08092F1038FEF8093F003E6CF45
:1028D0000E94AB0682E08093F1031092E60310920F
:1028E000E7031092E8031092E9038091FC039091B2
:1028F000FD039093FB038093FA0380912E048130B3
:1029000009F423C408F4D1C2823009F4F1C283303F
:1029100009F418C380912E048F5F837080932E0476
:102920000E94400550CE10910704111108C070E0BC
:1029300060E085E00E94920583E08093F10380913E
:102940000604811104C084E08093F103CECF81306E
:1029500061F6113051F68091E503882371F0809182
:10296000E403882381F370E060E085E00E94920533
:102970001092E3031092F103B8CF70E060E085E0BD
:102980000E94920583E0E0CF2091FC033091FD038B
:1029900080912704909128048217930718F40E94CD
:1029A0007508A3CF1092F10360E089E00E948304D0
:1029B0001092EA039ACF0E94CD0797CF8091E2034D
:1029C00081110BC080910704811130C01092E10386
:1029D00070E060E085E00E9492058091DF039091B5
:1029E000E003892B09F061C08091DD039091DE0343
:1029F0008035910508F059C08091EF038F3F81F534
:102A00008EE18093F1031092EB031092EC0310928D
:102A1000ED031092EE038091E1038F3F09F065CF43
:102A20008FE08093F1031092EF035FCF8091060453
:102A300081110CC08FEF8093E1031092EB03109291
:102A4000EC031092ED031092EE03C7CF8091E503E3
:102A5000882309F4BBCF8091E403882359F3BDCFC9
:102A60008091EB039091EC03A091ED03B091EE0304
:102A70000196A11DB11D8093EB039093EC03A093ED
:102A8000ED03B093EE031092F103409113045091C3
:102A9000140470E060E084179507A607B70708F4F0
:102AA000BACF84E18093F103B6CF88E2FBCF60E038
:102AB00089E00E9483042FB7F8948091C803909115
:102AC000C903A091CA03B091CB032FBF8093D90350
:102AD0009093DA03A093DB03B093DC038091290485
:102AE00090912A040A972091FC033091FD03281746
:102AF000390760F46091D80370E085E00E94920588
:102B000080EF8093EA039092F103D9CE70E060E009
:102B100085E00E9492051092EA031092F103CFCE55
:102B20008FB7F8944090C8035090C9036090CA03CF
:102B30007090CB038FBF4092D4035092D503609224
:102B4000D6037092D7030E94AB068091E5038823D9
:102B500011F1809107048823F1F08091D9039091BD
:102B6000DA03A091DB03B091DC03481659066A062C
:102B70007B0618F1B301A201481B590B6A0B7B0BB2
:102B80008091110490911204B0E0A0E04817590719
:102B90006A077B0790F04092D9035092DA03609263
:102BA000DB037092DC0370E060E085E00E94920538
:102BB0001092EA031092E103DDCE6091FC03709164
:102BC000FD038091290490912A040A96853333E00D
:102BD000930710F084E393E06817790740F070E002
:102BE00060E085E00E9492059092F1037ECE90E035
:102BF00080E04AE00E94EB0886E293E00E94DE0853
:102C00006091150470E0EDCF70E060E085E00E9417
:102C100092051092E20385E18093F10350CE61E0CA
:102C200089E00E9483042FB7F8948091C8039091A3
:102C3000C903A091CA03B091CB032FBF8093D003E7
:102C40009093D103A093D203B093D30382E08093F7
:102C5000E30386E18093F1030E94AB068FE080934B
:102C6000EA0343CE8FB7F8944090C8035090C9034D
:102C70006090CA037090CB038FBF4092D4035092F0
:102C8000D5036092D6037092D7030E94AB06809161
:102C9000D0039091D103A091D203B091D3034816F1
:102CA00059066A067B06F8F0A3019201281B390B2E
:102CB0004A0B5B0BDA01C90180349F41A105B105C4
:102CC00090F04092D0035092D1036092D203709260
:102CD000D30360E089E00E9483048FEF8093EF03C9
:102CE0001092F103BBCF86E18093F103B7CF10922E
:102CF000F1035ECE8FEF8093E2031092EF03A0907A
:102D0000CE03B090CF030091CC031091CD0370E0BF
:102D100060E085E00E9492056090DD037090DE0324
:102D2000E091DF03F091E003809124049091250469
:102D30006816790610F580911E0490911F048E1775
:102D40009F07D8F0C501B7010E94381B9B01C8013D
:102D5000B7010E94381BDB010E94ED181B012C01FA
:102D600020911C0430911D04A4E6B0E00E94ED18EF
:102D70006215730584059505A8F480912B04909144
:102D80002C04892B91F58AE28093F103EF2B09F44F
:102D900096CD1092EB031092EC031092ED0310927B
:102DA000EE038DCD20911A0430911B04A4E6B0E00F
:102DB0000E94ED182616370648065906C0F4809181
:102DC000200490912104E817F90788F480912204E7
:102DD000909123046816790650F4309741F0809161
:102DE0002B0490912C04892B71F689E2CDCF809130
:102DF000E403882341F28091E5038823B1F3109224
:102E0000F1031092EA03C2CF1092E6031092E70397
:102E10001092E8031092E9032091FC033091FD0326
:102E200080912704909128048217930708F0BACD67
:102E30000E94750813CF8091E6039091E703A0915B
:102E4000E803B091E903813E4EE29407A105B10584
:102E5000E0F42091290430912A042A50310940914C
:102E6000FC035091FD034217530778F40196A11D0E
:102E7000B11D8093E6039093E703A093E803B0931A
:102E8000E9030E94CD0780EFEACE8BE28093F10345
:102E90008FCD1092F10370E060E085E00E94920512
:102EA0001092E2030E94AB0683CD0091090410E06A
:102EB000000F111F86E10E945A0480959095817041
:102EC0009927082B0093090401110DC010920804E2
:102ED00088E10E945A048093070487E10E945A0403
:102EE0008093060417CD0F3F99F700930804F0CFA5
:102EF00081E00E94690683E00E946906BC0190E0BF
:102F000080E00E940F1A23E333E343E55BE30E9472
:102F1000C61A20E030E048EC52E40E94C61A20E0D5
:102F200030E048EC51E40E946E192AE037ED43E2AC
:102F30005CE30E946E190E94E01970930B04609389
:102F40000A04E8CC81E08983A0902B04B0902C0483
:102F5000BE016F5F7F4FC5010E94D0088091290498
:102F600090912A0412E0853353E0950730F411E084
:102F700022E0A216B10408F410E0BE016F5F7F4F9B
:102F80000E94D0088091270490912804853333E073
:102F9000930708F013E0BE016F5F7F4F0E94D008D7
:102FA000809126049FEF980F983C08F014E0BE0132
:102FB0006F5F7F4F90E00E94D00880912404909131
:102FC0002504873242E0940708F015E0BE016F5FE8
:102FD0007F4F0E94D0088091220490912304873271
:102FE00052E0950708F016E0BE016F5F7F4F0E9428
:102FF000D0088091200490912104893823E1920720
:1030000008F017E0BE016F5F7F4F0E94D0088091EB
:103010001E0490911F04893833E1930708F018E0EB
:10302000BE016F5F7F4F0E94D00880911C04909179
:103030001D04893542E0940708F019E0BE016F5F76
:103040007F4F0E94D00880911A0490911B0489350B
:1030500052E0950708F01AE0BE016F5F7F4F0E94B3
:10306000D00880911904853608F01BE0BE016F5F1F
:103070007F4F90E00E94D008809118048B3008F0B8
:103080001CE0BE016F5F7F4F90E00E94D0088091EE
:103090001704853108F01DE0BE016F5F7F4F90E09F
:1030A0000E94D00880911604853608F01EE0BE010B
:1030B0006F5F7F4F90E00E94D00880911504BE01A1
:1030C0006F5F7F4F90E00E94D00880911304909131
:1030D0001404813127E2920708F010E1BE016F5F0E
:1030E0007F4F0E94D008BE016F5F7F4F8091110417
:1030F000909112040E94D008BE016F5F7F4F8091B3
:103100000F04909110040E94D00880910D049091BA
:103110000E048436910508F413E1BE016F5F7F4F02
:103120000E94D008E981F0E0E050FE4F908180914C
:103130000C04981301C011110E945D0980912D04A7
:10314000893130F010922D041F9A0E94080CE2CBB6
:103150008F5F80932D04F9CF10922F0410923004CA
:103160001092310410923204DBCBF999FECF92BD5C
:1031700081BDF89A992780B50895262FF999FECF39
:103180001FBA92BD81BD20BD0FB6F894FA9AF99A84
:103190000FBE01960895A1E21A2EAA1BBB1BFD01CA
:1031A0000DC0AA1FBB1FEE1FFF1FA217B307E40726
:1031B000F50720F0A21BB30BE40BF50B661F771F7E
:1031C000881F991F1A9469F760957095809590955E
:1031D0009B01AC01BD01CF010895A29FB001B39F37
:1031E000C001A39F700D811D1124911DB29F700D10
:1031F000811D1124911D08955058BB27AA270E94B4
:1032000014190C94871A0E94791A38F00E94801AB7
:1032100020F039F49F3F19F426F40C94761A0EF43A
:10322000E095E7FB0C94701AE92F0E94981A58F366
:10323000BA17620773078407950720F079F4A6F59B
:103240000C94BA1A0EF4E0950B2EBA2FA02D0B0198
:10325000B90190010C01CA01A0011124FF27591BDB
:1032600099F0593F50F4503E68F11A16F040A22FE1
:10327000232F342F4427585FF3CF46953795279552
:10328000A795F0405395C9F77EF41F16BA0B620B51
:10329000730B840BBAF09150A1F0FF0FBB1F661F98
:1032A000771F881FC2F70EC0BA0F621F731F841FDB
:1032B00048F4879577956795B795F7959E3F08F001
:1032C000B0CF9395880F08F09927EE0F97958795C3
:1032D00008950E944C1A08F481E008950E94821912
:1032E0000C94871A0E94801A58F00E94791A40F0B4
:1032F00029F45F3F29F00C94701A51110C94BB1AF9
:103300000C94761A0E94981A68F39923B1F3552306
:1033100091F3951B550BBB27AA27621773078407E8
:1033200038F09F5F5F4F220F331F441FAA1FA9F37E
:1033300035D00E2E3AF0E0E832D091505040E6956C
:10334000001CCAF72BD0FE2F29D0660F771F881FCD
:10335000BB1F261737074807AB07B0E809F0BB0BC0
:10336000802DBF01FF2793585F4F3AF09E3F5105D4
:1033700078F00C94701A0C94BB1A5F3FE4F3983EFB
:10338000D4F3869577956795B795F7959F5FC9F7BD
:10339000880F911D9695879597F90895E1E0660F3E
:1033A000771F881FBB1F621773078407BA0720F0B7
:1033B000621B730B840BBA0BEE1F88F7E095089520
:1033C0000E94A01A88F09F5798F0B92F9927B751FB
:1033D000B0F0E1F0660F771F881F991F1AF0BA95B9
:1033E000C9F714C0B13091F00E94BA1AB1E0089543
:1033F0000C94BA1A672F782F8827B85F39F0B93F35
:10340000CCF3869577956795B395D9F73EF490956B
:103410008095709561957F4F8F4F9F4F0895E894E9
:1034200009C097FB3EF490958095709561957F4F0C
:103430008F4F9F4F9923A9F0F92F96E9BB279395BA
:10344000F695879577956795B795F111F8CFFAF4CA
:10345000BB0F11F460FF1BC06F5F7F4F8F4F9F4FFB
:1034600016C0882311F096E911C0772321F09EE859
:10347000872F762F05C0662371F096E8862F70E0BF
:1034800060E02AF09A95660F771F881FDAF7880F99
:103490009695879597F90895990F0008550FAA0BEF
:1034A000E0E8FEEF16161706E807F907C0F0121657
:1034B0001306E407F50798F0621B730B840B950B5A
:1034C00039F40A2661F0232B242B252B21F40895AF
:1034D0000A2609F4A140A6958FEF811D811D08954C
:1034E00097F99F6780E870E060E008959FEF80ECB7
:1034F000089500240A94161617061806090608955A
:1035000000240A9412161306140605060895092EBF
:103510000394000C11F4882352F0BB0F40F4BF2B2E
:1035200011F460FF04C06F5F7F4F8F4F9F4F08956E
:1035300057FD9058440F551F59F05F3F71F0479564
:10354000880F97FB991F61F09F3F79F08795089549
:10355000121613061406551FF2CF4695F1DF08C068
:10356000161617061806991FF1CF86957105610585
:1035700008940895E894BB2766277727CB0197F92D
:1035800008950E944C1A08F48FEF08950E94D91AEA
:103590000C94871A0E94791A38F00E94801A20F041
:1035A000952311F00C94701A0C94761A11240C9433
:1035B000BB1A0E94981A70F3959FC1F3950F50E0C3
:1035C000551F629FF001729FBB27F00DB11D639FD5
:1035D000AA27F00DB11DAA1F649F6627B00DA11D7B
:1035E000661F829F2227B00DA11D621F739FB00D21
:1035F000A11D621F839FA00D611D221F749F332791
:10360000A00D611D231F849F600D211D822F762F29
:103610006A2F11249F5750409AF0F1F088234AF006
:10362000EE0FFF1FBB1F661F771F881F9150504072
:10363000A9F79E3F510580F00C94701A0C94BB1AA8
:103640005F3FE4F3983ED4F3869577956795B795F9
:10365000F795E7959F5FC1F7FE2B880F911D969513
:10366000879597F908950E944C1A880B990B089535
:10367000AA1BBB1B51E107C0AA1FBB1FA617B70798
:1036800010F0A61BB70B881F991F5A95A9F78095B4
:103690009095BC01CD010895EE0FFF1F881F8BBFD1
:0C36A0000790F691E02D1994F894FFCFEC
:1036AC0000316253C4F5A697B988DBEA7D4C1F2E16
:1036BC004372211087B6E5D4FACB98A93E0F5C6D06
:1036CC0086B7E4D5427320113F0E5D6CFBCA99A8F6
:1036DC00C5F4A796013063527C4D1E2FB889DAEBE6
:1036EC003D0C5F6EF9C89BAA84B5E6D740712213D6
:1036FC007E4F1C2DBA8BD8E9C7F6A59403326150C6
:10370C00BB8AD9E87F4E1D2C02336051C6F7A495B5
:10371C00F8C99AAB3C0D5E6F4170231285B4E7D6A5
:10372C007A4B1829BE8FDCEDC3F2A1900736655495
:10373C0039085B6AFDCC9FAE80B1E2D34475261785
:10374C00FCCD9EAF38095A6B4574271681B0E3D275
:10375C00BF8EDDEC7B4A192806376455C2F3A09165
:10376C004776251483B2E1D0FECF9CAD3A0B586955
:10377C0004356657C0F1A293BD8CDFEE79481B2A45
:10378C00C1F0A3920534675678491A2BBC8DDEEF35
:10379C0082B3E0D1467724153B0A5968FFCE9DAC25
:1037AC000000000001033E0284024E03B5029302A6
:1037BC00A7025265736574212076657273696F6E0A
:1037CC0020342E3033000D0A005072657373696F0C
:1037DC006E206D6178205B6261725D203D20006E11
:0C37EC00616E00696E66006F766600007A
:00000001FF
